:100000000C94340018950000189500001895000015
:10001000189500001895000018950000189500002C
:10002000189500001895000018950000189500001C
:10003000189500001895000018950000189500000C
:1000400018950000189500001895000018950000FC
:1000500018950000189500001895000018950000EC
:1000600018950000189500008FEF8DBFC8EDE0ECEB
:100070004E2E88E08EBFD8E0F8E05F2EA89584B7BA
:10008000082E877F84BF88E1992780936000909332
:100090006000EEEFF7E0A0E0B1E088278D933197A4
:1000A000E9F787E68093C40080E08093C50088E18B
:1000B0008093C1000E940301662487E880937A0040
:1000C00080E480937C000E94F8008CE00E94510143
:1000D00070917A00706870937A0000917C00007FC4
:1000E00000937C000E948D01A0E0B1E08D939C9371
:1000F0000E94FD00E0E5F3E00E94EF000E94F600A0
:10010000A0E0B1E00D911C91083E53E0150718F0F6
:1001100011F00C948D000C949300EAE5F3E00E943A
:10012000EF000C94ED00A0E0B1E00D911C910835BA
:1001300052E0150718F011F00C94A0000C94A600E2
:10014000E2E6F3E00E94EF000C94ED00A0E0B1E0E5
:100150000D911C91003951E0150718F011F00C9425
:10016000B3000C94B900EAE6F3E00E94EF000C94AF
:10017000ED00A0E0B1E00D911C91083C50E01507A6
:1001800018F011F00C94C6000C94CC00E2E7F3E0F8
:100190000E94EF000C94ED00A0E0B1E00D911C91E5
:1001A000063450E0150718F011F00C94D9000C94A7
:1001B000DF00EAE7F3E00E94EF000C94ED00A0E01E
:1001C000B1E00D911C91043150E0150710F00C9432
:1001D000ED00E2E8F3E00E94EF000C946D000E9455
:1001E000A401802D11F057D0FACF089580EC59C0AA
:1001F00081E057D005D080E854C080E852D00895FF
:1002000083E099277BC08AEF90E00E947E01579A95
:10021000569A559A549A219A209A289885E090E007
:100220000E947E0129985F985E985D9A5C9A299A4F
:10023000EF93FF93ECE8F1E00E947201FF91EF91E0
:10024000299859D0299AEF93FF93ECE8F1E00E94A6
:100250007201FF91EF9129984ED0299AEF93FF9365
:10026000ECE8F1E00E947201FF91EF91299843D0F0
:100270005C98299AEF93FF93ECE8F1E00E947201F9
:10028000FF91EF91299837D088E20BD08EE009D00A
:1002900086E007D00895289A829505D004D02BD007
:1002A00008952898F9CF859510F45C9A01C05C9860
:1002B000859510F45D9A01C05D98859510F45E9A5D
:1002C00001C05E98859510F45F9A01C05F98299AE5
:1002D000EF93FF93ECE8F1E00E947201FF91EF9140
:1002E000299808953197F1F70895689462F8089570
:1002F000E89462F8089581E090E000C0EF93FF93E6
:10030000EE27E82BE92B31F0E0EAFFE03197F1F737
:100310000197D1F7FF91EF91089570917A00706481
:1003200070937A0000907A0006FCFCCF70917A00FE
:10033000706470937A0000907A0006FCFCCF809184
:100340007800909179000895C8953196002008951D
:100350006B65792076616C7565004E6F6E65202047
:10036000000053656C65637400004C4546542020C2
:100370000000446F776E2020000075702020202040
:0A0380000000726967687420000035
:00000001FF
